:0200000480007A
:100000006F000005732F2034930F80006308FF03F7
:10001000930F90006304FF03930FB0006300FF038E
:10002000130F000063040F0067000F00732F2034CC
:1000300063540F006F00400093E19153171F0000BD
:1000400023223FFC171F000023200FFC6FF01FFF2F
:100050009300000013010000930100001302000050
:100060009302000013030000930300001304000038
:100070009304000013050000930500001306000020
:100080009306000013070000930700001308000008
:10009000930800001309000093090000130A0000F0
:1000A000930A0000130B0000930B0000130C0000D8
:1000B000930C0000130D0000930D0000130E0000C0
:1000C000930E0000130F0000930F0000732540F102
:1000D0006310050097020000938202017390523072
:1000E000735044749702000093820201739052305F
:1000F00073500018970200009382020273905230EE
:10010000B70200809382F2FF7390023B9302F001EA
:100110007390023A7350403097020000938242017C
:100120007390523073502030735030309301000080
:1001300097020000938242ED739052301305100035
:100140001315F501634C05000F00F00F930110002B
:100150009308D0051305000073000000930200000F
:10016000638A020073905210B7B20000938292101B
:100170007390223073500030372500007320053013
:100180007350300097020000938242017390123442
:10019000732540F1730020309301200073D03000AC
:1001A0003715000013054523F315350093031000A0
:1001B000639C752693013000732530009303400340
:1001C00063147526930140007325100093034001CA
:1001D000631C752493015000735521009303100094
:1001E0006314752493016000732530009303400568
:1001F000631C752293017000737512009303400114
:100200006314752293018000732530009303000569
:10021000631C75209301A000B7150000938545234A
:1002200013060000D38005F4530106F45380202404
:10023000530500E4B7130000938343236316751E30
:100240009301B000B7150000938545231306F0FF16
:10025000D38005F4530106F453802024530500E4B1
:10026000B793FFFF938343236310751C9301C00072
:10027000B79500009385452313060000D38005F44D
:10028000530106F453802024530500E4B713000003
:1002900093834323631A75189301D000B795000028
:1002A000938545231306F0FFD38005F4530106F42C
:1002B00053802024530500E4B793FFFF9383432327
:1002C0006314751693014001B7150000938545230B
:1002D00013060000D38005F4530106F45390202444
:1002E000530500E4B793FFFF93834323631E751206
:1002F00093015001B7150000938545231306F0FFC5
:10030000D38005F4530106F453902024530500E4F0
:10031000B7130000938343236318751093016001A2
:10032000B79500009385452313060000D38005F49C
:10033000530106F453902024530500E4B793FFFFC4
:10034000938343236312750E93017001B7950000E8
:10035000938545231306F0FFD38005F4530106F47B
:1003600053902024530500E4B713000093834323E4
:10037000631C750A9301E001B715000093854523BE
:1003800013060000D38005F4530106F453A0202483
:10039000530500E4B71300009383432363167508E5
:1003A0009301F001B7150000938545231306F0FF74
:1003B000D38005F4530106F453A02024530500E430
:1003C000B793FFFF938343236310750693010002E5
:1003D000B79500009385452313060000D38005F4EC
:1003E000530106F453A02024530500E4B793FFFF04
:1003F00093834323631A750293011002B79500009B
:10040000938545231306F0FFD38005F4530106F4CA
:1004100053A02024530500E4B71300009383432323
:1004200063147500631030020F00F00F6380010049
:100430009391110093E111009308D00513850100F9
:10044000730000000F00F00F930110009308D00517
:100450001305000073000000731000C000000000CE
:10046000000000000000000000000000000000008C
:0C04700000000000000000000000000080
:1010000000000000000000000000000000000000E0
:1010100000000000000000000000000000000000D0
:1010200000000000000000000000000000000000C0
:1010300000000000000000000000000000000000B0
:081040000000000000000000A8
:040000058000000077
:00000001FF
